:100000000C945B000C9481000C9481000C94810092
:100010000C9481000C9481000C9481000C9481005C
:100020000C9481000C9481000C9481000C9481004C
:100030000C9481000C9481000C9481000C9481003C
:100040000C948E090C9481000C94DF0B0C948100AD
:100050000C9481000C9481000C9481000C9481001C
:100060000C9481000C9481008D09000000070002AF
:10007000010000030406000000000000000001026F
:100080000408102040800102040810200102040826
:100090001020040404040404040402020202020204
:1000A0000303030303030000232629000025282B54
:1000B000000024272A0011241FBECFEFD4E0DEBFAA
:1000C000CDBF14E0A0E0B1E0E2ECFDE102C005909C
:1000D0000D92A430B107D9F714E0A4E0B4E001C058
:1000E0001D92A63EB107E1F710E0CAE6D0E004C0D9
:1000F0002297FE010E94BF0EC836D107C9F70C94A3
:10010000BD080C940000CF93DF93CDB7DEB72497E2
:100110000FB6F894DEBF0FBECDBF24E0FE013196CE
:10012000DC01122E0E94C30E69817A818B819C8131
:1001300024960FB6F894DEBF0FBECDBFDF91CF91EE
:10014000089590931F0480931E0470931D04609380
:100150001C0450931B0440931A040E948300609374
:10016000340470933504809336049093370480915F
:100170001C0490911D040E948300609330047093CE
:100180003104809332049093330480911A04909147
:100190001B040E94830060932C0470932D048093B1
:1001A0002E0490932F0408958EE090EAA6E6BAE319
:1001B0008093040490930504A0930604B09307046D
:1001C0000895CF93DF93CDB7DEB724970FB6F89499
:1001D000DEBF0FBECDBF69837A838B839C83DA0138
:1001E00084E0FE013196182E0E94C80E24960FB6A8
:1001F000F894DEBF0FBECDBFDF91CF91089560931D
:10020000590470935A0480935B0490935C044CE00F
:1002100050E00E94E10008956091590470915A04E1
:1002200080915B0490915C040895609155047091F5
:1002300056048091570490915804089560910A04DF
:1002400070910B0480910C0490910D0408952F92ED
:100250003F924F925F926F927F928F929F92AF9256
:10026000BF92CF92DF92EF92FF920F931F93CF93A3
:10027000DF93CDB7DEB724970FB6F894DEBF0FBE7D
:10028000CDBF39014A010E94F10C7B018C016091C4
:100290003404709135048091360490913704A8019C
:1002A00097010E94110E69837A838B839C836093EC
:1002B00028047093290480932A0490932B0460915E
:1002C0003C0470913D0480913E0490913F04A8014C
:1002D00097010E94F20C5B016C0160933C047093E7
:1002E0003D0480933E0490933F042090300430906E
:1002F00031044090320450903304A201910160E037
:1003000070E088EC92E40E94340D7B018C019B012B
:10031000AC01C601B5010E94A40D181664F017FBCC
:10032000109517F91095A8019701C601B5010E9413
:10033000A10D882344F4E0923C04F0923D04009324
:100340003E0410933F0420913C0430913D044091C1
:100350003E0450913F04C201B1010E94110E5B01A5
:100360006C01609324047093250480932604909379
:100370002704209138043091390440913A04509177
:100380003B04C401B3010E94F10C9B01AC016091DC
:100390002C0470912D0480912E0490912F040E94C2
:1003A000110E7B018C0160932004709321048093D3
:1003B000220490932304609238047092390480924E
:1003C0003A0490923B04A601950169817A818B8160
:1003D0009C810E94F20CA80197010E94F10C2496C6
:1003E0000FB6F894DEBF0FBECDBFDF91CF911F9146
:1003F0000F91FF90EF90DF90CF90BF90AF909F90C4
:100400008F907F906F905F904F903F902F900895C6
:10041000EF92FF920F931F937B018C0120E030E05D
:1004200040E050E00E94A10D18165CF00F2EF0E0A5
:10043000EF2EF0E0FF2EF0E00F2FF0E01F2FF02D59
:1004400014C020E030E04AE754E4C801B7010E943C
:10045000A40D882354F00F2EF0E0EF2EF0E0FF2ED5
:10046000FAE70F2FF4E41F2FF02DE0924904F092E9
:100470004A0400934B0410934C041F910F91FF907A
:10048000EF90089561E086E00E94B30A08956091BC
:10049000490470914A0480914B0490914C04089552
:1004A0001F93182F682F86E00E941A0B10934804A0
:1004B0001F910895EF92FF920F931F930E94B3092B
:1004C0009B01AC01609344047093450480934604FF
:1004D00090934704E0904004F0904104009142045E
:1004E00010914304DC01CB018E199F09A00BB10BC5
:1004F000885E9340A040B04028F42E153F05400789
:10050000510798F481E00E94500280914404909138
:100510004504A0914604B091470480934004909311
:100520004104A0934204B0934304209144043091C9
:1005300045044091460450914704809140049091B5
:100540004104A0914204B0914304281B390B4A0B8B
:100550005B0B57FD05C0CA01B9010E94970D14C07D
:10056000CA01B9016170707080709070569547959E
:1005700037952795622B732B842B952B0E94970D13
:100580009B01AC010E94F20C2091490430914A0475
:1005900040914B0450914C040E94A40D88231CF000
:1005A00080E00E9450021F910F91FF90EF900895FC
:1005B0006091340470913504809136049091370431
:1005C00008956091300470913104809132049091CB
:1005D0003304089560912C0470912D0480912E04B1
:1005E00090912F04089560933404709335048093A0
:1005F00036049093370440911E0450911F040E94CA
:10060000E1000895609330047093310480933204C4
:100610009093330440911C0450911D040E94E1000A
:10062000089560932C0470932D0480932E0490936E
:100630002F0440911A0450911B040E94E100089578
:100640000F931F930DE514E040E052EC61E070E081
:10065000C8010E94CA0864E071E0C8010E94FD0858
:1006600067E471E0C8010E94FD0861E871E0C8011B
:100670000E94FD0864EC71E0C8010E94FD081F9112
:100680000F9108950F931F930DE514E060EF71E053
:10069000C8010E94FD0863E172E0C8010E94FD08E4
:1006A0006EE272E0C8010E94FD0860E572E0C801D8
:1006B0000E94FD0868E872E0C8010E94FD086DEA2A
:1006C00072E0C8010E94FD0868EC72E0C8010E9457
:1006D000FD0867ED72E0C8010E94FD086DEF72E051
:1006E000C8010E94FD0862E273E0C8010E94FD0893
:1006F00067E473E0C8010E94FD086CE673E0C8017E
:100700000E94FD081F910F9108952F923F924F92E2
:100710005F926F927F928F929F92AF92BF92CF9291
:10072000DF92EF92FF920F931F93CF93DF93CDB79A
:10073000DEB724970FB6F894DEBF0FBECDBF3B01E6
:100740004C015C834B8320E030E040E050E00E94AD
:10075000A10D88232CF460E070E080E09FEB04C0E2
:1007600060E070E080E09FE300E010E008C020E07F
:1007700030E040E251E40E94340D0F5F1F4F2B81A7
:100780003C81021713079CF39B01AC01C401B30128
:100790000E94F20C5B016C0120E030E040E050E090
:1007A000C401B3010E94A10D87FD0DC00F2EFDEC09
:1007B0002F2EFCEC3F2EFCEC4F2EFDE35F2EF02D98
:1007C0001A8219820CC0D7FAD094D7F8D094EECF01
:1007D0001701280189819A8101969A83898320E0F3
:1007E00030E040E251E4C201B1010E94110E7B01F0
:1007F0008C01A60195010E94A10D18164CF720E06E
:1008000030E040E050E0C401B3010E94A10D882314
:100810002CF46DE28DE594E00E94D908E981FA811B
:10082000EF2B51F42AE030E040E050E060E070E06F
:100830008DE594E00E945E098824992433C0A201CA
:100840009101C601B5010E94340D0E947A0D7B0111
:100850008C010027F7FC0095102F2AE030E0B8014A
:10086000A7018DE594E00E945E09C801B7010E94CE
:10087000970DA20191010E94110E9B01AC01C601CE
:10088000B5010E94F10C5B016C0120E030E040E218
:1008900051E4C201B1010E94340D1B012C010894E6
:1008A000811C911C29813A818216930644F28B8126
:1008B0009C8118161906ACF56EE28DE594E00E9455
:1008C000D9088824992420E030E040E251E4C601B0
:1008D000B5010E94110E5B016C010E947A0D7B0133
:1008E0008C010027F7FC0095102F2AE030E0B801BA
:1008F000A7018DE594E00E945E09C801B7010E943E
:10090000970D9B01AC01C601B5010E94F10C5B0182
:100910006C010894811C911CEB81FC818E169F0652
:1009200091F624960FB6F894DEBF0FBECDBFDF91CF
:10093000CF911F910F91FF90EF90DF90CF90BF90DC
:10094000AF909F908F907F906F905F904F903F906F
:100950002F900895EF92FF920F931F9380910804B8
:1009600090910904E0900E04F0900F04009110049F
:1009700010911104885E93401CF581E00E94440AA6
:10098000AA2797FDA095BA2FBC01CD010E94970D13
:100990009B01AC01C801B7010E94F20C60930E04E8
:1009A00070930F04809310049093110480910804B5
:1009B00090910904019690930904809308042AC039
:1009C00020910404309105044091060450910704DD
:1009D000C801B7010E94110E20E030E040E052E46F
:1009E0000E94F20C60930A0470930B0480930C0431
:1009F00090930D04109209041092080480E090E096
:100A0000A0E0B0E080930E0490930F04A093100434
:100A1000B09311041F910F91FF90EF9008950F93E1
:100A20001F930DE514E063E973E0C8010E94DD083F
:100A3000609128047091290480912A0490912B04DC
:100A400042E050E00E9485036DEA73E0C8010E9415
:100A5000DD08609124047091250480912604909112
:100A6000270442E050E00E94850361EB73E0C80177
:100A70000E94DD086091200470912104809122047D
:100A80009091230442E050E00E94850365EB73E0FF
:100A9000C8010E94DD086091490470914A04809168
:100AA0004B0490914C0440E050E00E9485036EEBB3
:100AB00073E0C8010E94DD081F910F9108950F9304
:100AC0001F930DE514E060EC73E0C8010E94DD089F
:100AD0006091590470915A0480915B0490915C0478
:100AE00042E050E00E9485036BEC73E0C8010E9475
:100AF000DD086091550470915604809157049091DF
:100B0000580442E050E00E94850367ED73E0C8019D
:100B10000E94DD08609134047091350480913604A0
:100B20009091370442E050E00E94850362EE73E04A
:100B3000C8010E94DD0860913004709131048091F9
:100B400032049091330442E050E00E94850366EE47
:100B500073E0C8010E94DD0860912C0470912D049F
:100B600080912E0490912F0442E050E00E94850372
:100B70006AEE73E0C8010E94DD0860910001709187
:100B80000101809102019091030142E050E00E9436
:100B9000850364EF73E0C8010E94DD086091490499
:100BA00070914A0480914B0490914C0440E050E0D5
:100BB0000E9485036EEF73E0C8010E94DD081F915B
:100BC0000F910895EF92FF920F931F936091590434
:100BD00070915A0480915B0490915C0442E050E073
:100BE0000E94850301E014E0FDE5EF2EF4E0FF2E06
:100BF000B801C7010E94DD08609155047091560448
:100C0000809157049091580442E050E00E9485037F
:100C1000B801C7010E94DD08609134047091350469
:100C2000809136049091370442E050E00E948503A1
:100C3000B801C7010E94DD08609130047091310451
:100C4000809132049091330442E050E00E94850389
:100C5000B801C7010E94DD0860912C0470912D0439
:100C600080912E0490912F0442E050E00E94850371
:100C7000B801C7010E94DD086091490470914A04DF
:100C800080914B0490914C0440E050E00E94850319
:100C9000C7010E94E5081F910F91FF90EF90089502
:100CA000CF93DF9385C18DE594E00E94D3089093A4
:100CB00019048093180482359105C1F460E070E056
:100CC00080EF91E40E94F30260E070E080E090E049
:100CD0000E94020360E070E080E090E00E94110357
:100CE00060E070E088E493E40E94FF0080911804C3
:100CF0009091190480359105A1F4609134047091AC
:100D00003504809136049091370420910001309190
:100D1000010140910201509103010E94F20C0E94D6
:100D2000F302809118049091190480379105A1F481
:100D300060913404709135048091360490913704A9
:100D40002091000130910101409102015091030175
:100D50000E94F10C0E94F3028091180490911904F2
:100D600089349105A1F4609130047091310480912F
:100D7000320490913304209100013091010140919F
:100D80000201509103010E94F20C0E940203809123
:100D900018049091190489369105A1F460913004EA
:100DA00070913104809132049091330420910001BC
:100DB0003091010140910201509103010E94F10C18
:100DC0000E940203809118049091190484349105C3
:100DD000A1F460912C0470912D0480912E049091C7
:100DE0002F042091000130910101409102015091A6
:100DF00003010E94F20C0E9411038091180490914B
:100E0000190484369105A1F460912C0470912D048D
:100E100080912E0490912F042091000130910101C6
:100E200040910201509103010E94F10C0E941103B4
:100E3000809118049091190484359105A1F4609172
:100E4000590470915A0480915B0490915C04209144
:100E500000013091010140910201509103010E9473
:100E6000F20C0E94FF0080911804909119048437BD
:100E70009105A1F46091590470915A0480915B042A
:100E800090915C0420910001309101014091020198
:100E9000509103010E94F10C0E94FF00C0911804C0
:100EA000D0911904CB32D10521F5609100017091E8
:100EB0000101809102019091030120E030E040E2C5
:100EC00051E40E94110E6093000170930101809320
:100ED00002019093030120E030E048EC52E40E94CC
:100EE000A40D18160CF03FC080E090E0A8ECB2E42E
:100EF00025C0CD32D10559F56091000170910101F5
:100F0000809102019091030120E030E040E251E441
:100F10000E94340D609300017093010180930201DF
:100F2000909303012AE037ED43E25CE30E94A10DB8
:100F30008823CCF48AE097EDA3E2BCE38093000120
:100F400090930101A0930201B09303010CC0C53737
:100F5000D10549F490E080911704882309F491E0C9
:100F60009093170410C0C736D10549F490E08091E2
:100F70001604882309F491E09093160404C0A09706
:100F800011F40E945F058091180490911904CF9785
:100F900011F40E9442038091180490911904823642
:100FA000910531F40E940F058DE594E00E94E5085B
:100FB0008DE594E00E94CF08882309F074CE0E944A
:100FC000B3092091120430911304409114045091FC
:100FD0001504621773078407950740F410921204F2
:100FE0001092130410921404109215040E94B30975
:100FF000209112043091130440911404509115046F
:10100000621B730B840B950B693C7105810591057F
:10101000C8F028533F4F4F4F5F4F20931204309337
:1010200013044093140450931504809117048823EB
:1010300049F080911604882319F00E94E20502C04D
:101040000E945F05DF91CF9108950E9450060E9493
:10105000AA0480910A0490910B04A0910C04B09111
:101060000D048093550490935604A0935704B093B5
:1010700058040E94B30920914D0430914E044091D0
:101080004F0450915004621773078407950740F48A
:1010900010924D0410924E0410924F04109250047E
:1010A0000E94B30920914D0430914E0440914F04A9
:1010B00050915004621B730B840B950B693C7105B6
:1010C0008105910540F128533F4F4F4F5F4F2093CB
:1010D0004D0430934E0440934F045093500420919C
:1010E0005504309156044091570450915804609132
:1010F000590470915A0480915B0490915C040E94A1
:101100002701609351047093520480935304909389
:1011100054040E9408020E945A02089548E050E0D8
:1011200064E070E080E090E00E94A1008CE090E03C
:101130000E9483006093590470935A0480935B0467
:1011400090935C040E94B30960934D0470934E0425
:1011500080934F04909350040E9442020E94200307
:101160008EE090EAA6E6BAE3809304049093050427
:10117000A0930604B09307040895CFEFD4E0DEBF38
:10118000CDBF0E94FA090E948E080E942508FDCF5B
:1011900008950895CB01BA010E94650B08950E943D
:1011A000A60B992708950E94B70B08950E94D60BAD
:1011B0000895862F0E941D0C0895CB010E94240CD7
:1011C0000895862F0E941D0C08950F931F938C0184
:1011D0006DE00E94D9086AE0C8010E94D9081F91F9
:1011E0000F9108950F931F938C010E94D908C80195
:1011F0000E94E5081F910F9108950F931F938C0192
:101200000E94DD08C8010E94E5081F910F91089512
:101210000F931F938C010E94E108C8010E94E5080A
:101220001F910F910895CB01BA0133274427552709
:101230000E94310C08952AE00E94130908950F932B
:101240001F938C010E941B09C8010E94E5081F9191
:101250000F910895AB01662777270E941B09089517
:10126000EF92FF920F931F93CF93DF93EC017A01DC
:101270008B0177FF0BC06DE20E94D9081095009595
:10128000F094E094E11CF11C011D111D2AE0B8014D
:10129000A701CE010E941309DF91CF911F910F91F9
:1012A000FF90EF9008950F931F938C010E943009D7
:1012B000C8010E94E5081F910F910895211531057D
:1012C00021F4642F0E94D90808952A30310519F4B9
:1012D0000E94300908950E94130908950F931F93E7
:1012E0008C010E945E09C8010E94E5081F910F91C0
:1012F0000895AB01662757FD6095762F0E9430094F
:1013000008950F931F938C010E947909C8010E94D0
:10131000E5081F910F910895089508951F920F9267
:101320000FB60F9211248F939F93AF93BF93809129
:10133000620490916304A0916404B09165040196E5
:10134000A11DB11D8093620490936304A093640473
:10135000B0936504BF91AF919F918F910F900FBE95
:101360000F901F90189560916204709163048091B2
:1013700064049091650427E0660F771F881F991F0A
:101380002A95D1F72DE730E040E050E00E946C0E46
:10139000CA01B9010895AF92BF92CF92DF92EF9246
:1013A000FF920F931F935B016C010E94B3097B01B5
:1013B0008C010E94B3096E197F09800B910B6A158D
:1013C0007B058C059D05A8F31F910F91FF90EF9071
:1013D000DF90CF90BF90AF900895019751F0880FA4
:1013E000991F880F991F02972FB7F8940197F1F76B
:1013F0002FBF0895789410926204109263041092A3
:1014000064041092650484B5826084BD84B58160F3
:1014100084BD85B5826085BD85B5816085BDEEE6FC
:10142000F0E0808181608083E1E8F0E0808182608B
:101430008083808181608083E0E8F0E0808181604A
:101440008083E1EBF0E0808184608083E0EBF0E07A
:10145000808181608083ECE7F0E080818F778083FA
:10146000808180648083EAE7F0E08081846080830B
:1014700080818260808380818160808380818068B8
:1014800080831092C100089590917C00907F8F70AE
:10149000982B90937C0080917A00806480937A00EE
:1014A00080917A0086FDFCCF2091780080917900B0
:1014B0009927982F88273327822B932B08951F93E2
:1014C000CF93DF93182FEB0161E00E94B30AE12F65
:1014D000FF27E659FF4F8491833051F480918000BB
:1014E000806880938000D0938900C093880037C0C3
:1014F000843051F480918000806280938000D0938A
:101500008B00C0938A002BC0813029F484B5806899
:1015100084BDC7BD24C0823029F484B5806284BDF7
:10152000C8BD1DC0863041F48091B00080688093B2
:10153000B000C093B30013C0873041F48091B00075
:1015400080628093B000C093B40009C0C038D10558
:1015500014F460E001C061E0812F0E941A0BDF915A
:10156000CF911F910895282F3327C90182589F4F8B
:10157000FC0194912E563F4FF9018491882381F00C
:10158000E82FFF27E055FF4FE491FF27662329F45A
:10159000808190958923808308958081892B808321
:1015A0000895482F5527CA0186599F4FFC01249161
:1015B000CA0182589F4FFC0194914E565F4FFA0129
:1015C00034913323A1F1222331F1233021F480918E
:1015D00080008F7705C0243031F4809180008F7DAA
:1015E0008093800018C0213019F484B58F7704C02F
:1015F000223021F484B58F7D84BD0DC0263021F4C6
:101600008091B0008F7705C0273029F48091B00019
:101610008F7D8093B000E32FFF27EA55FF4FE491C1
:10162000FF278081892319F081E090E0089580E010
:1016300090E00895482F5527CA0186599F4FFC0115
:101640002491CA0182589F4FFC0194914E565F4FDE
:10165000FA0134913323C1F1222331F1233021F4F3
:10166000809180008F7705C0243031F48091800014
:101670008F7D8093800018C0213019F484B58F7756
:1016800004C0223021F484B58F7D84BD0DC0263086
:1016900021F48091B0008F7705C0273029F4809124
:1016A000B0008F7D8093B000E32FFF27E555FF4FFB
:1016B000E491FF27662329F4808190958923808314
:1016C00008958081892B80830895EF92FF920F9374
:1016D0001F937B018C0122E030E040E050E00E944B
:1016E0008E0E205C3D4B404F5F4FCA01B901A801EF
:1016F00097010E948E0E2150304040405040BB2741
:1017000057FDBA95A52F942F832F2F5F3F4F4F4F33
:101710005F4F8093C50021502093C400E1ECF0E0BE
:1017200080818061808380818860808380818068FF
:1017300080831F910F91FF90EF900895982F8091D3
:10174000C00085FFFCCF9093C6000895809160048F
:101750009091610420915E0430915F04821B930B91
:1017600080589F4F60E870E00E94590E08954091A4
:101770005E0450915F04809160049091610484172D
:10178000950719F48FEF9FEF0895FA01EA59FB4F7F
:101790002081CA01019660E870E00E94590E909382
:1017A0005F0480935E04822F9927089580915E04E0
:1017B00090915F04909361048093600408951F9258
:1017C0000F920FB60F9211242F933F934F935F9375
:1017D0006F937F938F939F93AF93BF93EF93FF93F9
:1017E0004091C600E0916004F0916104CF01019640
:1017F00060E870E00E94590E9C0180915E04909117
:101800005F042817390739F0EA59FB4F40833093BA
:10181000610420936004FF91EF91BF91AF919F917C
:101820008F917F916F915F914F913F912F910F9089
:101830000FBE0F901F90189508950E949E0B08955B
:101840008AE00E941D0C0895CF93DF93EC0103C042
:1018500021960E941D0C88818823D1F7DF91CF91BA
:1018600008952F923F924F925F926F927F928F9244
:101870009F92AF92BF92CF92DF92EF92FF920F931F
:101880001F93CF93DF93CDB7DEB7A0970FB6F89431
:10189000DEBF0FBECDBF6B017C0119012A016115AE
:1018A00071058105910521F480E30E941D0C4BC058
:1018B0006624772443015E010894A11CB11C8501B4
:1018C000060D171DC701B601A20191010E946C0E01
:1018D000F80160830894611C711C811C911CC70174
:1018E000B601A20191010E946C0E69017A012115D5
:1018F00031054105510519F773010894E108F10814
:10190000EA0CFB1CAA24BB24650111C0F7018081ED
:101910008A3010F4805D01C0895C0E941D0C08941F
:10192000A108B108C108D1080894E108F108882786
:101930009927DC0186199709A809B909A816B906DB
:10194000CA06DB0619F7A0960FB6F894DEBF0FBEE5
:10195000CDBFDF91CF911F910F91FF90EF90DF905E
:10196000CF90BF90AF909F908F907F906F905F903F
:101970004F903F902F900895EF92FF920F931F93F7
:101980007B018C0197FF0BC08DE20E941D0C10950E
:101990000095F094E094E11CF11C011D111D2AE05A
:1019A00030E040E050E0C801B7010E94310C1F91C7
:1019B0000F91FF90EF90089520E130E040E050E07B
:1019C0000E94310C089528E030E040E050E00E9491
:1019D000310C089522E030E040E050E00E94310CEC
:1019E00008955058192EEFD001D0D2C0BA1762070F
:1019F000730784079507B1F188F40EF410940B2E49
:101A0000BA2FA02D062E622F202D072E732F302DDA
:101A1000082E842F402D092E952F502DFF2755235A
:101A2000B9F0591B49F0573E98F0469537952795E0
:101A3000A795F0405395C9F776F0BA0F621F731F50
:101A4000841F30F4879577956795B795F040939507
:101A500017FA0F2E0895BF1BBB27BA0B620B730B2F
:101A6000840BF6CFDEF6DBC0AED001D091C055239B
:101A700059F0992369F09F575F57951B33F442F44F
:101A8000903811F4915805C09BC091589F3F09F4BC
:101A9000C6C0BB27112462177307840730F4660F92
:101AA000771F881FBB1F915098F311D00F920FD052
:101AB0000F920DD0A0E82617370748071B0609F03C
:101AC000A048BA2F602D7F918F9100240895A0E83F
:101AD0000024621773078407B10528F0621B730B9B
:101AE000840BB1090A2A660F771F881FBB1FA695B2
:101AF00081F7089597FB73D09F3738F0FEE9F91B03
:101B0000982F872F762F6B2F05C086C096958795C7
:101B100077956795F150D0F73EF490958095709544
:101B200061957F4F8F4F9F4F0895E89403C097FBB7
:101B30000EF4F3DFB62F672F782F892F9EE900244C
:101B400027C00ED05EF004C00BD026F001C008D034
:101B500019F020F48FEF089580E0089581E0089552
:101B600097FB092E052600F8689430D0E89407FC0E
:101B700007C0621773078407950721F008F40094E3
:101B80000794989408959A95BB0F661F771F881F36
:101B900011249923A1F08823B2F79F3F59F0BB0F7E
:101BA00048F421F4002011F460FF04C06F5F7F4F00
:101BB0008F4F9F4F881F9795879597F908952CC051
:101BC0009FEF80EC0895052E092607FA440F551F54
:101BD0005F3F79F0AA27A51708F051E04795880FD5
:101BE000991F9F3F31F0BB27B91708F091E0879507
:101BF00008959F919F911124E3CF97FB880F991F20
:101C00009F3F31F0BB27B91708F091E08795089501
:101C10009F919F911124D4CF6627772788279927F2
:101C20000895D1DF01D0B4CF992339F0552329F09D
:101C30009F575F57950F13F49AF1F1CF91589F3F3B
:101C4000E1F3629FA12D0F92BB27639FA00DB11DF1
:101C5000EE27729FA00DB11DEE1FAF93AA27649FC0
:101C6000B00DE11D739FB00DE11DAA1F6627829F75
:101C7000B00DE11DA61F5527749FE00DA11D551F36
:101C8000839FE00DA11D561F849FA00D511D852F20
:101C90007A2F6E2F1F900F9088231AF4939539F4A2
:101CA0008FCF000C111CBB1F661F771F881F0128D8
:101CB000089597FB092E07260AD077FD04D049D056
:101CC00006D000201AF4709561957F4F0895F6F7BD
:101CD000909581959F4F0895A1E21A2EAA1BBB1BD8
:101CE000FD010DC0AA1FBB1FEE1FFF1FA217B307E8
:101CF000E407F50720F0A21BB30BE40BF50B661FFE
:101D0000771F881F991F1A9469F7609570958095C1
:101D100090959B01AC01BD01CF01089597FB092E61
:101D200005260ED057FD04D0D7DF0AD0001C38F4AA
:101D300050954095309521953F4F4F4F5F4F0895F7
:101D4000F6F790958095709561957F4F8F4F9F4FD7
:101D50000895AA1BBB1B51E107C0AA1FBB1FA617F2
:101D6000B70710F0A61BB70B881F991F5A95A9F744
:101D700080959095BC01CD010895EE0FFF1F059051
:101D8000F491E02D099409D001921A94E1F7089595
:101D900001900BD01A94E1F70895F999FECFB2BDE6
:101DA000A1BDF89A119600B40895F999FECFB2BD7D
:101DB000A1BD00BC11960FB6F894FA9AF99A0FBE1D
:021DC000089584
:101DC2000000803F0A57656C636F6D6520746F2059
:101DD20074686520424243432C2074686520426146
:101DE200726520426F6E657320436F66666565207B
:101DF200436F6E74726F6C6C657220666F722041F5
:101E0200726475696E6F0053656E64206261636B04
:101E1200206F6E65206F72206D6F7265206368613E
:101E22007261637465727320746F20736574757068
:101E32002074686520636F6E74726F6C6C65722EAD
:101E4200004966207468697320697320796F75721E
:101E520020696E697469616C2072756E2C20706CD9
:101E62006561736520656E74657220275227207440
:101E72006F20526573657420746865204545505221
:101E82004F4D2E00456E74657220273F2720666FE6
:101E9200722068656C702E20204865726527732059
:101EA200746F206120677265617420637570210010
:101EB20053656E642074686573652063686172613E
:101EC200637465727320666F7220636F6E74726FD3
:101ED2006C3A003C73706163653E203A207072690F
:101EE2006E7420737461747573206E6F7700752041
:101EF2003A20746F67676C6520706572696F6469F8
:101F02006320737461747573207570646174650005
:101F120067203A20746F67676C652075706461741E
:101F220065207374796C65206265747765656E20CF
:101F320068756D616E20616E642067726170686998
:101F42006E67206D6F64650052203A20726573657A
:101F5200742F696E697469616C697A6520504944AD
:101F6200206761696E2076616C7565730062203A44
:101F7200207072696E7420504944206465627567EE
:101F82002076616C756573003F203A207072696E2D
:101F9200742068656C70002B2F2D203A2061646AD2
:101FA2007573742064656C746120627920612066A7
:101FB2006163746F72206F662074656E00502F70BB
:101FC200203A2075702F646F776E2061646A757392
:101FD200742070206761696E2062792064656C7478
:101FE2006100492F69203A2075702F646F776E2047
:101FF20061646A7573742069206761696E20627911
:102002002064656C746100442F64203A2075702F3F
:10201200646F776E2061646A7573742064206761EF
:10202200696E2062792064656C746100542F74209B
:102032003A2075702F646F776E2061646A757374CD
:10204200207365742074656D702062792064656CFC
:1020520074610050494420666F726D756C6120286E
:1020620050202B2049202D2044293A2000202B20CB
:1020720000202D200020504F5745523A20002000CA
:10208200205345542054454D503A002C204355527C
:102092002054454D503A002C204741494E53207060
:1020A2003A0020693A0020643A002C2044656C749E
:1020B200613A20002C20506F7765723A2000200A86
:0420C200002C2000CE
:00000001FF
